:10000000002C0020F5280000F1280000F128000055
:1000100000000000000000000000000000000000E0
:10002000000000000000000000000000F1280000B7
:100030000000000000000000F1280000F12800008E
:10004000F1280000F1280000F12800006D0E0000EA
:10005000F1280000F1280000F1280000451F0000F1
:10006000F1280000F1280000F1280000F12800002C
:10007000F1280000F1280000F1280000F12800001C
:10008000F1280000F1280000F1280000F12800000C
:10009000F1280000F1280000F1280000F1280000FC
:1000A000F1280000F1280000F1280000F1280000EC
:1000B00010B5064C2378002B07D1054B002B02D03E
:1000C000044800E000BF0123237010BD1C01002084
:1000D000000000006432000008B5084B002B03D07C
:1000E0000748084900E000BF07480368002B03D019
:1000F000064B002B00D0984708BDC046000000000A
:100100006432000020010020643200000000000082
:10011000EFF3108072B6BFF35F8F034B00221A70AB
:10012000434258417047C04614010020024B1A78E0
:10013000013AD2B21A707047CC030020044B1A78EF
:10014000013AD2B21A701B78024B00221A70704723
:1001500042010020D2030020002070470020704799
:1001600010B50F4B0F4C0020207018800E4BA122B1
:100170001A7020225A7002220C4958809880DA8026
:100180001881E1235B020B600823087148718B71B1
:10019000074B9847237801200133DBB2237010BD51
:1001A00066060020CC030020D80300203801002080
:1001B0002D30000008B500200149024B984708BDCA
:1001C000380100202D300000002805D0034B01220B
:1001D0001A70BFF35F8F62B67047C04614010020EB
:1001E000124B60211A7850B20A40002809DA002028
:1001F000202A1AD15A78212A17D1DA88072A14D14D
:100200000FE00020202A10D15A78202A04D0101C98
:1002100022384242504108E0DA88072A05D10449D1
:10022000196104499A819960012070476C09002086
:10023000B501000038010020F7B5364B1A78002AC6
:1002400066D1354CA047354D2C8800280FD0344B53
:10025000984784425CD0334B9847334A334B1478E9
:10026000071CE4B26100C95A002919D101E0304BE2
:10027000EEE7304E28493388013333808847002821
:1002800006D13388632B03D8381C2B4B98473FE0AB
:10029000214A9047002803D03288284B9A42F3D94C
:1002A000244B00221A80264B1B78934205D16342CF
:1002B00063411D49DBB20B7002E063425C41E4B272
:1002C000144A01231370381C1B4B9847174B6700C7
:1002D000DE5B413EFF3E731E9E41F6B2002E09D00A
:1002E0000D498847002801D00D4B00E0104B98477E
:1002F000288000E02E800D49A20124021419CB5B56
:10030000104A1149121900918120311C0F4CA0474D
:10031000F7BDC046D4030020C5140000D003002060
:10032000D914000011010000430100204401002005
:10033000C914000040010020C90100001F03000093
:1003400065060020480100205D03000055170000ED
:1003500008B5014B984708BD3902000008B50028D0
:100360000CD1074B1A7853425A41064B5200D052D7
:10037000054B1870054B1870054B984708BDC046D3
:10038000430100204401002065060020D403002022
:100390003902000010B5074B9847074A074B1B88E6
:1003A0001178074A49008C5AE41A064B9847201CDA
:1003B00010BDC04611010000D3030020CE03002071
:1003C000C8030020C901000008B5034B9847431E2D
:1003D0009841C0B208BDC04695030000F0B5194B66
:1003E00085B098471849194A0C781578E4B2EDB2EF
:1003F000002D08D1164E670033880393154BFB5A26
:10040000039FBB4203D9144B9847002018E0358066
:1004100066426641F6B20E700F4F01261670B8475D
:100420000E4B281C9847A2010D4B240214190D4AAB
:100430000093A02312190220311CB3400A4CA0479C
:1004400005B0F0BD11010000D303002064060020B8
:10045000CE030020C8030020C9010000C90300002A
:10046000F1040000E40300205517000038B5134BD9
:10047000134D00242C701C70124B1C70124B1C70FE
:10048000124B1C805C80124B1C80124B9847124B05
:100490001C70124B1C70124B1C80124B1C80124B98
:1004A0009847A04209D02B780133DBB22B702B7810
:1004B000DBB2012B01D10D4A137038BDD4030020EB
:1004C0004201002065060020430100204401002075
:1004D000D00300203902000064060020D30300206E
:1004E000C8030020CE030020DD030000D20300205B
:1004F00013B500281CD10F4B1B785C426341DBB263
:1005000000290ED199011B02CB180B49101CCB18E6
:100510000A491A1C0091A02301218B40084CA047D6
:1005200006E0084A5B009952074B1870074B984742
:1005300013BDC046D3030020E4030020F1040000F3
:1005400055170000C803002064060020DD030000EA
:1005500008B50020014B984708BDC046C9030000FC
:10056000F7B5194B00269B79093B5A425341DBB240
:100570000193164B9847164B164F3C881D78164B27
:100580009847EDB2154B6A00D35AA4B2A34205D8DE
:10059000134B1878C0B20028EBD113E0AB012D0249
:1005A0005D19104B2D19EB5C01341E43A4B20E4BA8
:1005B0003C809847019B002B03D000233602019317
:1005C000D7E7301CFEBDC0463801002011010000F5
:1005D000D3030020CE030020C9010000C80300207F
:1005E000D2030020E4030020DD03000038B5114BE6
:1005F0009847114A114B1178C9B24C00E45AA02314
:100600005B009C420FD10E4B1B78002B0BD10D4D84
:100610002B78DBB2002B06D101242C704C426141B7
:10062000C9B211701C1C084B9847A0204000001B49
:1006300038BDC046110100004301002044010020E4
:10064000D403002065060020C901000008B5034B53
:100650009847431E9841C0B208BDC046ED05000052
:1006600008B50020014B984708BDC0464D06000064
:10067000F8B5154B0C1C9D79093D6B425D41EDB2FF
:100680000020124B9847002805D1114B1878C0B2B2
:100690000028F5D117E00F4B98470F4B0F491B78F7
:1006A000DBB25E00725A571C775299011B02CB18BD
:1006B0000B499A180B4B54549847002D02D0241222
:1006C0000025DDE70120F8BD380100204D060000BF
:1006D000D20300201101000043010020440100204A
:1006E00048010020C901000008B5011C014B002091
:1006F000984708BD7106000008B5034B58887F2352
:100700001840024B984708BD6C090020D51800001E
:1007100030B5144B1A7800239A4221D0124B1B6833
:100720001B681A79824201D8002319E00F4A13602E
:10073000DC789D7824022C431C199C420ED95D78EC
:10074000042D08D19D78854205D1DD788D4202D1F6
:100750001360012304E01D785B19EEE71360E3E703
:10076000181C30BD710600206806002074060020A9
:10077000094B1B681B68DA78997812020A439B18A8
:1007800002788018834205D94278042A02D0052ACB
:10079000F6D100E0002070476806002038B5104B05
:1007A000051C9847002801D1002018E00D4B1C685B
:1007B000201C0D4B9847041E0AD06279237912023F
:1007C0001A438078E178094B98470028F0D1EBE78D
:1007D000074BAD001B685B68EB581B68984738BD3A
:1007E0001107000074060020710700003D1500008D
:1007F00068060020F8B500210F4F051CB847041EFD
:1008000018D00E4BAA001B685B68D658F36898474F
:10081000011C281CB847041E0CD0094B1D68281C5D
:10082000084B9847051E03D08078074B9847F6E79A
:1008300073689847201CF8BD110700006806002067
:100840007406002071070000E914000008B5014B90
:10085000984708BDA119000038B50C4B00241A7840
:100860001D1CA24205D100232B70094B01221A80C6
:1008700038BD084B1B681B681B79A342F3D9201CA9
:10088000054B01349847E4B2F3E7C04671060020F7
:100890006E06002068060020F507000008B5024B30
:1008A0009847024B984708BD051A000059080000F8
:1008B00010B50B4B00241B78A3420FD0094B1B68CB
:1008C00019680A79A24209D95B68A200D3581B694A
:1008D000002B00D098470134E4B2EFE710BDC046CA
:1008E0007106002068060020F8B5A44C0023A381FF
:1008F00023616361237858B2002803DAE288002A72
:1009000000D1B2E16021194000D065E11F2200282A
:1009100000DBA9E0E588002D00D15DE1134067D13F
:100920006378062B09D0082B5DD0002B00D053E153
:10093000022D00D050E1924892E06088050A022D15
:100940000CD006D8012D00D046E18E4B18680178F6
:1009500040E0032D1FD00F2D13D03DE1894BC0B2D5
:1009600019684A7C824200D836E15B68C000C058F2
:10097000C178837809021943834B9847A268557060
:100980002AE0804B9868002800D125E1C17883785F
:10099000090219431EE0C0B2032800D91CE102F08D
:1009A00051FB070004000A0061011D21774A04E0A1
:1009B000774804210EE0774A0A21002376485D003B
:1009C000D65C451901336E80DDB28D42F6D3490005
:1009D000023101706C4B9847E388A2899A4200D893
:1009E000CAE0A381C8E0012D00D0F5E06B4837E0F4
:1009F000012B25D163780A2B00D0EDE0012D00D02A
:100A0000EAE0664B1B78002B00D1E5E0644B2679C9
:100A10001F683A681379B34200D8DDE0301C614B9F
:100A20009847051E00D1D7E07B68B600F358DB6815
:100A300098475D4B01211870181C534B984799E05B
:100A4000022B00D0C8E06378002B00D0C4E0022D58
:100A500000D0C1E0554B20799847554B1880181CA1
:100A6000291C494B984787E013404DD160780138E5
:100A7000082800D9B0E002F0DBFA0CAFAFAF05AF49
:100A8000AFAF1A00E388002B00D0A5E0494B2361EB
:100A900072E0E388002B00D09EE06388012B00D039
:100AA0009AE0374B02211A888A431A8064E0E5886D
:100AB000002D00D090E0404B9847002800D18BE0FB
:100AC000304EA27831684B7C9A4200DD84E03B4B8B
:100AD0009847A378314A1370002B4DD03849304ADB
:100AE0005B187168DB00CB181360161C33681B6839
:100AF0001B79AB4240D9281C0021324B9847002873
:100B00006AD00135EDB2F1E7012B15D163780B2BDB
:100B100062D1E388002B5FD1204B1B78002B5BD088
:100B20002579294B281C66889847002854D0F1B2B3
:100B3000281C244B98471CE0022B4DD16378012BD5
:100B400002D0032B09D047E0E388002B44D163880F
:100B5000002B41D120791D4B0AE0E388002B3BD1CB
:100B60006388002B38D12079194B98472079194B8D
:100B70009847051C002D2FD0012077E06C0900203C
:100B80006E060020A0000020F518000033000020B1
:100B90009000002028000020540000207106002052
:100BA00068060020110700007006002009160000EA
:100BB0006C060020F9060000E51800005908000046
:100BC000FFFFFF1F9D070000F50700001917000039
:100BD000891400001D16000022781F231340012BEA
:100BE0001ED1234B1B78002B1AD0224B25791E686F
:100BF00032681379AB4213D9281C00211E4FB84725
:100C000000280DD07368AA00D658F3689847011CD5
:100C1000281CB847002803D0B36898470028ABD1F8
:100C200022781F231340022B1FD1114B00241B7865
:100C3000002B1AD00F4B1B6819680A79A24214D9ED
:100C40005B68A200D558E96888470B4B011C201C43
:100C50009847002809D0AB68984700288CD1013408
:100C6000E4B2E7E70421054AA7E60020F8BDC04644
:100C700071060020680600201107000026320000DF
:100C80000368987AC009704770B50C4B0822056854
:100C9000041CDA67201C0A4EB0470028FAD12B88C2
:100CA000022293432B8020756075201CB0470028DA
:100CB000FBD12B88012213432B8070BD04E100E09F
:100CC000810C0000F8B50668071C0D1C141C381CAC
:100CD0000F4B98470028FAD13A79002A0AD01A23F4
:100CE000012A12D11723012C0FD80634A400A551D4
:100CF000031C0AE01723022C07D806498D4204D8AA
:100D00000C34ADB26400A553131C181CF8BDC046CA
:100D1000810C0000FFFF0000F7B52D4B0160151C92
:100D20009A6920210A439A6101A90223041C0B70CD
:100D30000420284B98470420274B9847274B201C1A
:100D40009847AB7823712B796371254B1C602B88F6
:100D500026683380AB78002B16D01720012B36D1B4
:100D600033889BB23380EB78002B03D0338880220A
:100D700013433380201C1B4B9847021EFAD1201CC2
:100D8000A968194B984719E033880422134333802C
:100D9000EB781720002B1AD1201C124FB847021EE7
:100DA000FAD1201CA968104FB847201C0D4B98475A
:100DB0000028FAD1201CE9680122B8472B790020CD
:100DC000834204D072888023DB0113437380FEBD0D
:100DD000000400400128000079270000890C000071
:100DE00040070020810C0000C50C000070B503799D
:100DF000041C05680E1C1520002B05D1201C034B7C
:100E000098470028FAD1AE8270BDC046810C000020
:100E1000031C022A0CD00079002805D0012805D136
:100E20001720012A0FD803E0022A01D917200AE06F
:100E3000901C8000C1500120197D9040021C0A4383
:100E4000D2B21A750020704710B5036880220229BB
:100E500003D001228A4003242240DA710122437D1B
:100E60008A40111C1943C9B2417510BD38B5114BE8
:100E70001B68597D1C681A7D207A0A40E17901407F
:100E8000C80906D0510701D51B69984780232372F2
:100E90000EE00125294203D02A4208D09B6805E0D4
:100EA0000225294204D02A4201D0DB6898472572E6
:100EB00038BDC04640070020EFF3108072B6BFF384
:100EC0005F8F034B00221A70434258417047C0465F
:100ED000140100200F2303405B00C00918180238DA
:100EE00014235843014B18187047C0467C06002055
:100EF000F0B58E7985B072B20D1C544B301C002AAF
:100F000046DA98470F2737400197028AC368029252
:100F10006D88041CED188368C560877C9D4221D0D4
:100F20005E1B4B4AB6B2964206D94A4B101C029938
:100F30009847474B5E1AB6B20023BA0706D5464B10
:100F4000301C029998478BB25A4253415A00A37CF5
:100F500002218B4313436268A37452193F480199DD
:100F6000331C0AE0B807C00F0AD0022362689F430F
:100F70003A480199A77452190023394CA04763E0FD
:100F800001239F432368A774002B5DD0291C59E0DF
:100F900098470F2333400293038A041C0193837CF8
:100FA0002F885A0710D5C268436801999B1803938C
:100FB0008068294B98470A1C02992A4B01398901FC
:100FC000C9180398284B9847E368FA18A368E260A9
:100FD0009A4200D9E360AA88BA422AD1E5689D42C4
:100FE00027D05E1B1A4FB6B2BE4206D9381C194B29
:100FF000019998477F1ABBB205E0301C164B019946
:101000009847761AB3B2019A1448184E93420BD2FD
:10101000A37C04221343029AA374013A114B920158
:10102000D2180299019B02E0626802995219B047F6
:101030000AE0A37C01229343A3742368002B03D00E
:10104000E1680020321C984705B0F0BDD50E0000C5
:10105000FF1F0000A1310000E13000000408002063
:101060006D1E00004407002005320000B91E00007C
:1010700010B5064B064C05221A70201C8021054B2A
:101080009847201C0021044B984710BDF70600200C
:1010900004080020F31D00000D1E000037B51E4B94
:1010A000041C9847226801AD80239372281C1B4BB7
:1010B000984703236B70291C201C194B9847201C50
:1010C0001849194B9847194D201C00210222184B32
:1010D000A84700210A1C201C164BA847164B201CB1
:1010E00000210122A847154D201C00210222A847FB
:1010F00000210A1C201CA847201C00210122A8470F
:1011000023680F4A19890A408021C9000A431A81BD
:101110000C4B00221A7037BD59080000111C00004A
:10112000211C000084090020011F0000A91A0000F2
:10113000951200004916000085110000F91A000000
:10114000FFF3FFFFF706002010B5084B084C032201
:101150001A70201C0749084B9847084B00219A68D1
:10116000201C0B1C064CA04710BDC046F7060020F3
:101170000408002084090020011F00006C090020E1
:101180006D1E000008B589790C4B4AB2002A08DAB6
:101190001B78012B02D10A4B98470DE0042B0BD191
:1011A00007E01A78022A02D104221A7004E0032A06
:1011B00002D10448044B984708BDC046F7060020FA
:1011C0004911000004080020F31D0000F8B51D4D72
:1011D0001D4E2B88B4891D4FE41AA4B2002C1BD1DC
:1011E0001B4A11885B189BB21380F2889A4203D085
:1011F000184B1B78002B07D0174B04221A70381C91
:101200001649174B98471CE07369002B0BD0984781
:10121000002808D02C80B4893F2C04D90D4B002223
:101220001A70402402E00B4B01221A702B88B2681E
:10123000381CD2180021231C0A4EB0472B88E41812
:101240002C80F8BDF40600206C0900200408002062
:1012500078060020F8060020F70600208409002008
:10126000011F00006D1E000008B5014B984708BD26
:10127000B1080000064B9A8C910605D4D968D0229B
:101280000A40D02AFAD102E0DA68D106FCD57047CC
:101290000008004070B5274E0C1C3378002B06D098
:1012A000254B1B69002B00D09847002333702388FF
:1012B000082B01D0214B2DE0214C1F4D23782B70A2
:1012C00063786B70E378A2781B02D3186B80637924
:1012D00022791B02D318AB80E379A2791B02D318C1
:1012E000EB80184B98470028E4D02B787F2B0DD942
:1012F000154B00211980154B221C198002233370D5
:1013000013484023134CA047134B03E0EB88002BFA
:1013100002D1124B98470BE00B4B002119800B4B6D
:10132000221C19800123337009484023094CA0472F
:1013300070BDC046F70600206C0900207110000047
:1013400084090020E908000078060020F406002047
:1013500004080020B91E0000CD1100004911000052
:10136000002805D0034B01221A70BFF35F8F62B6CD
:101370007047C04614010020F7B501AE114B041CA4
:101380001149301C04229847104B1D78A54217D0F4
:10139000002C08D00E4B375D98470E4BDA5D0132BA
:1013A000DA550D4B9847002D08D0094B755D9847CD
:1013B000084B5A5D013A5A55074B9847034B1C702E
:1013C000F7BDC046053200002B320000F6060020B3
:1013D000B90E0000380700206113000038B5084C32
:1013E000084D201C0621A847201C0421A8470221E3
:1013F000201C054B98470220044B984738BDC04637
:10140000040800208D1A00006D1A000079130000F6
:1014100038B50B4B98470B4C0B4B201C02219847BF
:101420000A4D201C0421A847094A0A4B201C06210A
:1014300098470621201CA8470320074B984738BD32
:1014400075120000040800208D1A00006D1A0000BB
:10145000DD1300004D1A00007913000010B5064C92
:101460000421201C054B98470221201C044B98475F
:101470000120044B984710BD040800208D1A00007D
:101480006D1A00007913000038B5041C211C0A48AD
:101490000A4B98470A4B201C9847827C031CD107B3
:1014A00008D501201D6882439A74002D02D0D968A6
:1014B000221CA84738BDC04604080020A91D000012
:1014C000D50E000000207047024B1B68188A80046C
:1014D000400D704704080020024B1B68188A80B238
:1014E0007047C04604080020F7B501AD041C0D4B41
:1014F000281C9847201C0C4B98470C4F0026291C91
:10150000381C0B4BEE702C7098470F21321C214079
:10151000381C084B9847381C321C211C064B984736
:10152000F7BDC046111C000089140000040800200B
:10153000211C0000D11A0000851B0000F7B501AC8A
:10154000061C294B201C0F1C151C984726700023D5
:10155000082D1DD90123102D1AD90223202D17D9AA
:101560000323402D14D90423802D11D980235B003F
:101570009D4201D805230BE080239B009D4201D8AA
:10158000062305E0194B9D4201D900202AE00723DC
:101590006370301C164B98470323391C0582194091
:1015A000012901D1022304E0022902D00329ECD150
:1015B0000423104DE370211C281C0F4B9847041E78
:1015C000E3D10F21221C0D4B3140281C0C4FB84792
:1015D000221C311C0B4C281CA047281C311C01224A
:1015E000A0470120FEBDC046111C0000FF03000003
:1015F000D50E000004080020211C0000F10E0000A0
:10160000A91A0000F91A000008B5011C014B024894
:10161000984708BDD51D0000040800200F2310B511
:101620000340041C0020032B07D80448211C044B52
:101630009847201C034B9847012010BD0408002048
:10164000F31D000089140000F8B5284E3378012BF3
:101650003FD1274A274C0D881788A3897A199342CE
:1016600001DADD1BADB2A3682349D8192A1C234B2C
:10167000EF199847BBB21E4F3B80402D05D1204D3E
:10168000E1882A88D218914208DCA3816369002B83
:1016900002D0984700280AD01A4B1DE0A2899A422E
:1016A00010D16069002802D08047002804D10523AA
:1016B0003370154B984718E03A882B88D3182B8045
:1016C00000233B8000210C4A4023104C1048A047C7
:1016D0000BE0022B02D10F4B984706E0054B1B692C
:1016E000002B00D0984700233370F8BDF706002088
:1016F000F40600206C090020840900200532000057
:1017000078060020491100001D160000B91E0000D7
:1017100004080020CD1100000F2370B50340061C03
:101720000024032B0ED8084B9847084B051C311C8E
:1017300007489847AB7C0124DA0703D5A343AB7471
:101740002B689847201C70BDD50E00000D1E0000B0
:1017500004080020F0B51E1C0F2385B00340071CB1
:10176000029103920193032B01D9002596E04D4B82
:101770009847051EF9D14C4B381C98474B4B041C1D
:101780009847A27CD10702D5494B984786E00123B0
:101790001A43A274002804D0464A1370BFF35F8F27
:1017A00062B60023E3600A9B039A0298A17C23603F
:1017B00001236260184002229840914301430420B3
:1017C0008143A17479B2A660002930DA002E1AD0C4
:1017D000394DB6B2AE4205D9218A281C374B9847FD
:1017E0006E1AB6B202990023994206D0344B218A70
:1017F000301C98478BB25A4253415A00A37C0221B5
:101800008B43134304E00299002909D0A37C93433E
:10181000A3740199039A331C2A4C2B48A0473AE041
:10182000A27C9A43A2740A9A002A08D10CE0002EE6
:101830000CD1A27C0A999A43A274002904D00020FA
:10184000011C3A1C0A9B9847012527E01A4FB6B2A3
:10185000258ABE4206D9381C184B291C98477F1A86
:10186000BBB205E0301C164B291C9847761AB3B260
:101870001548164EAB420BD2A37C04221343019AA7
:10188000A374013A124B9201D21801992B1C01E06A
:101890000199039AB04745424541EDB2281C05B075
:1018A000F0BDC04609160000D50E0000B90E0000BC
:1018B0006113000014010020FF1F0000A13100008F
:1018C000E13000006D1E000004080020B91E000079
:1018D00044070020024B80221B6810439872704717
:1018E00004080020024B1B68987A7F231840704739
:1018F00004080020014B9860998170476C09002012
:1019000008B5044B01201B681A8902431A81024B57
:10191000984708BD0408002079130000F8B503209B
:10192000164B9847164C01272368164E1A89201C1F
:10193000BA431A810421144AB047201C0021134ADB
:10194000B047391C201C124AB047124A201C022101
:10195000B047114D201C0421A847201C0021A84796
:10196000391C201CA847201C0221A8470B4A201C18
:101970000621B047201C0621A847F8BD79130000B6
:10198000040800204D1A00005D14000069120000D8
:101990009D100000111400006D1A0000DD130000FE
:1019A00073B50E4B984701AC061C0D4B201C984795
:1019B0000C4D00230C49221CA370281C0B4B98478C
:1019C000281C0B4B98470B4B984701200A4B984714
:1019D0000A4B9847301C0A4B984773BDB90E00005C
:1019E000552100000408002000500041652100003E
:1019F000311F000075120000791300001D1900004E
:101A00006113000010B5074B98470020064B98471C
:101A1000064B9847064B041C9847201C054B9847DB
:101A200010BDC0460119000079130000B90E000076
:101A3000391A000061130000034B1A78002A01D004
:101A400000221A707047C046F90600200B1C2E3386
:101A50009B001A50044AAA235B004900895AC25AC3
:101A60000A43C2520020704730320000064B490042
:101A70000268CB5A9383AB225200815A1943815298
:101A8000026800201383704730320000054BAB2200
:101A900052004900CB5A815A994381520268002072
:101AA000938270473032000010B58C00A418343493
:101AB000A4000419411863605931044BFF310878C0
:101AC0009B5C03430B70002010BDC0463E320000FB
:101AD00010B58C00A418031C34345B18A40004193E
:101AE0000449002059336060FF33895C1A788A43C7
:101AF0001A7010BD3E32000070B50F230B40C418A1
:101B000061341F4DFF342678AD5C35432570002AC3
:101B10000ED10268002B02D1FF3203230FE05B01DC
:101B2000D31849B2FF330222002926DB012224E028
:101B3000012A0FD10268002B03D1FF320C239372CC
:101B40001CE05B01D31849B2FF330822002914DBE3
:101B5000042212E0022A05D102685B01D318FF3388
:101B600010220AE0032A09D102685B01D31849B2A6
:101B7000FF334022002900DB20229A72002070BD32
:101B80003E32000070B50F230B40C4181F4D613466
:101B9000FF34AE5C2578B5432570002A0ED102686B
:101BA000002B02D1FF3203230FE05B01D31849B2AF
:101BB000FF330222002926DB012224E0012A0FD173
:101BC0000268002B03D1FF320C2353721CE05B012F
:101BD000D31849B2FF330822002914DB042212E093
:101BE000022A05D102685B01D318FF3310220AE0F4
:101BF000032A09D102685B01D31849B2FF3340229E
:101C0000002900DB20225A72002070BD3E32000005
:101C100000230370437083700123C370704700007A
:101C2000F0B5021C0D78C8780F232B40ED0904286D
:101C300000D998E0146801F0FBF90308495D7A00C7
:101C400008335B010020E054A9E05D016419FF3412
:101C500066781C20770700D0A1E0677870263742AD
:101C600000D09CE011206070146808335B01E0181C
:101C7000402444711268D31880221A718A78484B24
:101C8000002A08D05A195468802000060443546082
:101C90005469204307E05A195068400040085060DA
:101CA00050694000400850615D194C78686807220F
:101CB0003C4B1440184024072043686049780A4090
:101CC000696912070B4013436B6162E058012418E5
:101CD000FF34002D07D0677870261C2037425ED174
:101CE0006078202612E066781C20770757D160784C
:101CF00002262FE058012418FF34002D10D06778F9
:101D000070261C2037424AD16078302630436070FC
:101D100010681A1C0832520182188020107122E0CB
:101D200066781C2077073AD16078032612E05801C4
:101D30002418FF34002D07D0677870261C20374206
:101D40002DD160784026E1E766781C20770726D100
:101D5000607804263043607010681A1C0832520103
:101D60008218402050715B005D190D4B48782D01A1
:101D70005B19072210405C680A4A000722400243B0
:101D80005A608878002806D05968802212060A43D3
:101D90005A60002003E05A68520052085A60F0BDB1
:101DA000C4090020FFFFFF8F0F230B400268083398
:101DB0005B0149B2D218002905DA8021117102684D
:101DC000D318022204E0402151710268D318012285
:101DD000DA7170470F220A400368083252019B18DB
:101DE00049B29879002901DA800600E0C006C00FE8
:101DF00070470F220A4003680832520149B29B180B
:101E00002022002900DB10225A71704730B50F22C2
:101E10000A404CB201685301C918FF31CD79002C3A
:101E200011DA2024254220D04C710168CB18FF33F1
:101E30001C7A40210C4218D01972036808325201F2
:101E40009A18022310E0102425420ED04C7101682C
:101E5000CB18FF331C7A20210C4206D0197203687C
:101E6000083252019A180123137130BD70B50D1C50
:101E7000046808356D012E5D1C247606760F14D09B
:101E80000B4C490161180A610C1C0A4A49690A4055
:101E900062619A046369920C9B0B9B031343636119
:101EA000036800245D1980236B71201C70BDC0463F
:101EB000C4090020FF3F00F0F0B50D1C0468083590
:101EC0006D012E5D1C24770713D00B4C49010A517C
:101ED00061184C689A04094B1209234013434B6064
:101EE0004B6800249B0B9B034B6003685D194023E8
:101EF0002B71201CF0BDC046C4090020FF3F00F03C
:101F0000094B0A4A196059680A40802189020A432C
:101F10005A605A68920B92035A6003684022FF335A
:101F200000205A717047C046C4090020FF3F00F0EE
:101F3000036802211A780A431A7002689378022B08
:101F4000FCD07047F0B57E4C85B0206802681378ED
:101F5000DB0900D0F2E0118C8FB2002F4CD1AB2303
:101F60005B00C65A958BAA235B00ADB2C35A2E40C4
:101F70001E40744B7A00D35A1D4202D02268126868
:101F800093831E420FD07049062F06D16F4B1A89DA
:101F9000802312095B0013400B603B1C20682E332A
:101FA0009B001B5898470137072FE2D1C6E01E1C43
:101FB0000836B025009674016D00C618751959369B
:101FC0001419FF36B4460294E4792E7803956546D9
:101FD0002D78E4B22E40351C60262540344212D1C3
:101FE000102634422AD10C2634423AD1A60776D1A3
:101FF0000133082B00D1A1E03C1C1C410125D9B2C2
:102000002C42F5D0D3E75C011219FF32167A402436
:10201000264204D0147280225242114304E0167A00
:102020002024264202D01472494A9171602215423E
:1020300000D183E01B01C318DC337CE0029F0399CD
:10204000FE710A78324279D040495A018A185268A2
:102050001B0192043E49C318920CD8330A805B6876
:102060006BE05C011219FF32177A082637421DD047
:102070001672364A1419A67E02221834164202D06D
:10208000A6789643A670802252421143304A91713D
:10209000009902684F01D719FA7994074ED40C229F
:1020A00015424BD01B01C318D43344E0167A0427E1
:1020B0003E42F4D01772254A1219967A0224083249
:1020C000264202D09678A6439670214A91710099D3
:1020D00002684F01D719FA79D407E0D52EE05C01E8
:1020E0001219FF32177ABC46664602273E420CD0D0
:1020F000802617727642164A3143917113490C19A2
:1021000061698904890C518010E0177A01263742F1
:102110000CD016720E4A91710C490C196168890431
:10212000890C118061680901890C9180AF0705D085
:102130000D331B01C3185B680549984705B0F0BD16
:102140000C07002030320000FC060020C4090020EB
:102150000407002000220123027043708270C370C4
:1021600070470000F7B5171C634A00231360634AE9
:10217000051C1060624A29600C1CD169202001AE48
:1021800001430120D16106227370B070F3701820F2
:102190005C4B311C3270984706205A4A3070311C13
:1021A00019209047BB786846037069460620564B55
:1021B0009847564B062098472378012213432370F3
:1021C000A378D807FCD452490B685A0B1F231A4036
:1021D0009A4200D105221A409001268D4D4A324084
:1021E000024322850868820C13401F2B00D11D2357
:1021F000208D1F2213409043034323850B68072241
:10220000DB0D1340934200D103231340218D1A03A9
:10221000414B42480B401343238521783A787F2372
:10222000D2010B401343237079780123194023789E
:102230000422890093430B4323706062FB78012BD7
:1022400004D12B680C211A898A4306E0002B05D1A2
:102250002B680C241989A1430A431A818022304B30
:102260000021520098470023E918002204334A60F5
:10227000202BF9D1A918002310324B628B62CB625C
:102280000B63802AF6D12A1CA43213705370E9180C
:10229000081C0022A630AE31013302700A70082BF0
:1022A000F5D1131CE918B831002204330A601C2B45
:1022B000F8D1A918081C0023D430E0311032036093
:1022C000436083600B60802AF3D1AA225200AB5294
:1022D000AB225200AB52AC20EA1840001118613218
:1022E0000020FF32013308701070082BF3D10D4B22
:1022F00080221A60FEBDC046000700200C070020A7
:10230000000400409D2800000128000079270000FB
:10231000246080003FF8FFFFFF8FFFFFC40900200B
:102320001732000000E100E0094B196800290BD1C9
:10233000EFF31080074A002805D172B6BFF35F8F14
:1023400005490870012111701A6801321A6070473E
:10235000100700201407002014010020084B1A6801
:10236000013A1A601B68002B09D1064B1B78002B21
:1023700005D0054B01221A70BFF35F8F62B670471C
:10238000100700201407002014010020F7B50023D7
:1023900001AC144E80270125A370211CBF0211201F
:1023A000114B657025709847B761211C11200E4BA9
:1023B00025709847B761211C9836082723200A4BBF
:1023C000257098473760211C1B20074B25709847C4
:1023D000002337600F202370211C034B6570984742
:1023E000F7BDC04600440041ED23000007B5802240
:1023F00001AB1A700A785A704A789A708A78191C58
:10240000DA70014B984707BD9D28000010B50C4BB2
:1024100002211A680A431A60196880229143094A06
:1024200089B29184101CC168064ACC06FBD5996814
:102430000020D162596891621B689BB2938410BDE1
:10244000180700200008004070B50D4B45781E6A43
:10245000817804780122402086431540AD01301C6C
:102460000A402843D10180229043021C0A430548B8
:1024700003212140090202400A431A6270BDC0468E
:1024800000080040FFFCFFFF30B5027A4389920646
:102490009B059B0D120C1A43124B5A60428881888F
:1024A000C4791143827922430A434178C9010A431E
:1024B0001A600278042A0BD1047BC189058A0A4874
:1024C000A40609042C43014021439960196806E0E1
:1024D000202A06D1028A9A6019688422D2000A430F
:1024E0001A6030BD180700200000FF0308B5082857
:1024F00028D800F09DFD122727100B18051E21007B
:10250000114B02211A6A0A431A6204E00E4B02219F
:102510009A690A439A61002015E00B4B02211A8A3E
:102520000A431A82F7E7084B02219A8A0A439A82E1
:10253000F1E7064B984706E0054B02211A780A435B
:102540001A70E8E7172008BD000800400D240000BD
:1025500044080040F0B5C223344EDB00B360344B76
:102560001E215A688BB08A4304210A435A6005A889
:102570000023438083714370072303733F2320228A
:10258000C3812C4B02701A68920E3F2A00D11F2281
:10259000294B2A491B689B059B0D8B4200D1284B78
:1025A00043810823C37180235B008380254B027223
:1025B0000382254B984701A8012300258370234BF4
:1025C000457005709847224B06209847214B984745
:1025D00002AC0323211C65702572657223700220F2
:1025E00020231D4D6360A84702201C4FB8471C4B99
:1025F00098472A1CF1680D4BC806FBD5998C8020A2
:1026000001439984174B002507211D72281C5D7218
:102610009D7201232170211C6360237265706572B5
:102620009047281CB8470BB0F0BDC04600080040DA
:10263000004000412460800028608000FF0300000B
:10264000FF01000080BBFFFF892400004924000037
:10265000ED240000752600009526000039270000B3
:102660000D24000000040040014B5878C009704759
:10267000000C0040054B08219A690A439A61044BFB
:1026800001221A701A78D107FCD470470004004068
:10269000000C0040F8B50C784B782402051C061C91
:1026A0000443002B02D08023DB021C434B7A002B17
:1026B00002D080231B031C434B68012B13D95E1EE1
:1026C0001E400222002E09D19A4202D20136520047
:1026D000FAE7360280232E435B0303E01E028023C9
:1026E0002E439B021C430B7A002B02D080239B03BA
:1026F0001C430C4FB8470028FBD10B4B98470B4BA2
:102700001D70B8470028FCD1094DAE60B8470028BD
:10271000FCD16A6880235B0213401C436C60054B4C
:102720009847F8BD6926000029230000080C0040E6
:10273000000C00405D23000038B5051C094CA04783
:102740000028FBD1084B9847084B1D70A047002874
:10275000FCD1074B8022596852020A435A60054B4C
:10276000984738BD6926000029230000040C00406A
:10277000000C00405D23000010B5074B041C984777
:10278000064B80221C70064BD20159880A435A809E
:10279000044B984710BDC04629230000020C00409E
:1027A000000C00405D23000038B50F4B041C984717
:1027B0000E4B0F4A1C700F4B598858880905104062
:1027C00058805C880C48090F20405880101C5C8899
:1027D000084A6504FBD45388090203400B43538025
:1027E000064B984738BDC04629230000020C004024
:1027F000FFF0FFFF000C0040FFBFFFFF5D23000064
:1028000010B50C78034B240204439847024BA4B242
:102810005C8010BDA9270000000C004030B5D478C2
:1028200000239C421AD11478802C03D080232406E4
:102830005B02234354780225AC4309D19478002CE1
:1028400002D18024A40201E0C024E40223434160B9
:102850005478013C012C01D80F4C2340A0248DB2A8
:10286000E4052C431C438462D0240D0C24062C4325
:102870001C438462D478002C0CD15C0305D593787A
:10288000012B01D1816100E041615378013B012BB3
:1028900000D8816030BDC046FFFFFBFF08B5031CB8
:1028A0000A1C4009D90903D10549C001401800E0BC
:1028B00000201F210B4001219940024B984708BD81
:1028C000004400411D2800007047000008B5044B7B
:1028D0009847044B9847044B9847044B984708BDCA
:1028E000552500008D230000C9280000C9280000DC
:1028F000FEE700001148124910B5884201D00023BC
:1029000001E0104B07E0104CCA18A242F9D2C4589B
:1029100004331460F7E70D4A191D043B934203D2B8
:1029200000221A600B1CF6E7094A0A4B7F218A43F2
:102930009A60094B9847094B9847FEE764320000BC
:1029400000000020200100201C010020FC0B0020C2
:102950000000000000ED00E0B9310000652F00002C
:1029600008B51D4B1A6802321A601968FA22520122
:10297000914209D9194A1A4908201368C867997AF7
:1029800049B200290BDAFAE718683221154B98474B
:10299000002920D18022144B9202DA611BE01988B1
:1029A000022081431980136880221A720F4AC023C3
:1029B00008215B00D1500E4B984772B6BFF35F8F72
:1029C0000C4B00221A70BFF34F8F0B4A0B4BDA608F
:1029D000BFF34F8FFEE708BD34070020C40A002074
:1029E00004E100E0E13000000044004100E100E0CB
:1029F0009D080000140100200400FA0500ED00E02D
:102A000008B5074B08221A60064B98470028FBD0F0
:102A1000054B08221A600020044B9847C0B208BD3D
:102A200098440041510500009444004161050000B4
:102A3000084A80231B0570B5041C9361151C1E1CDD
:102A4000054B98470028FBD06E61201C034B98472C
:102A500070BDC0460044004161060000E906000068
:102A60000B4B0C4A1968914211D91A68D2B2002A4C
:102A700009D01A68012152085200494211801A688F
:102A800002321A60F1E7044B1B7DDA07FBD5704771
:102A900018010020FF3F00000040004110B50B1C52
:102AA00000225C1AA4B2844203D21C780133624033
:102AB000F7E7101C10BD0000F0B5944BC9B0587971
:102AC0006946087001381C2800D9F8E000F0B0FA17
:102AD0000F5A32F7F75DF7F7F7F7F7F7F7F7F7ADB4
:102AE00053869EC2F7F7F7F7F7F725F76B00002339
:102AF0004B7008238B704123CB7056230B715223EC
:102B00004B7149238B715323CB7150230B725F237D
:102B10004B7232238B720B24D2E05A7A00234B7013
:102B200002218A1A7A49D2006E461141B170F370BF
:102B30000424C5E09B7900224A70902B10D006D85F
:102B4000802B0BD0812B11D102238B7011E0912BA4
:102B500009D0922B0AD105238B700AE0012306E0ED
:102B600003248C70ACE004238B7002E000236946E0
:102B70008B700324A4E000234B70664A664B1A60F6
:102B800002249DE000234B70FAE79979DA7909066F
:102B900012040A43597A1B7A0A431B021A435F4BF9
:102BA00052001A602EE0597A002230290DD16E466B
:102BB000DB7AF1700221CB1A5549DB0019417270A2
:102BC000B27032717171B27106E068464270827003
:102BD000C170027142718271072471E08022D201BA
:102BE0004F4B197D188B2021FF3101431983910828
:102BF0004900D9614B4901321980FF328023DB0241
:102C00009A42EDD1002369464B70B9E79879DA7999
:102C10004249000210180C68434A80B2944208D816
:102C20000B68C018414B0860984700236A465370F0
:102C3000A6E70F3300228242F2D25D780C681E783C
:102C400014192D02640875196400ADB22580023292
:102C50000233F0E79879DB790002304A18186E46A3
:102C6000002381B27370304D1668CC1CA4B2AE4202
:102C70001DD98B4212D21568981C5D196D086D0024
:102C80002D886E463554156800AE5B195B085B00F5
:102C90001D8833182D0A5D70031CEAE7136800A82D
:102CA000C91803191160013B00221A7008E0834221
:102CB000F4D000AEF518FF26AE700133F7E700241C
:102CC0001B4D1B20A8471B4B260A1F78381CA84702
:102CD000F0B2A8471B235F4067407E40E0B2F7B2E6
:102CE000A8470E204740A8470026B3B2A34204D20B
:102CF0006946885DA8470136F7E769460E4B201CF8
:102D000098474740F8B2A84749B0F0BDDC0A002018
:102D100001981E004C1D00003407002018010020FF
:102D20000040004102A5FFFFFF3F0000612A0000B4
:102D3000312A0000320700209D2A0000F8B5002744
:102D40003D1C3C1C1F4B98471F49061C485501352C
:102D5000062CF7D8201C00F06BF904080C11171C86
:102D600023001B2E28D00025ECE7184B02241E70F0
:102D7000E8E7174B36021E800324E3E7144B0424D4
:102D80001A8816431E80DDE70E2E17D10027052472
:102D9000D8E70F4B01371B889F42D3D10624D1E7D8
:102DA000013DA8B20B4B98470025B04207D10A4B12
:102DB0001D600A4B9847F8BD0124C3E700252C1C71
:102DC000C0E7C046012A0000DC0A002032070020CC
:102DD000300700209D2A000034070020B92A000097
:102DE000094B0421DA690A43DA61084B2022198B66
:102DF000FF320A431A831A7DD10703D559681E2270
:102E00000A405A607047C04600040040004000413C
:102E10007FB500236A46164CD370138093700293DB
:102E20000393012313711349134B201C134E98472E
:102E300008222368326021688A7A52B2002AFBDBBA
:102E40001A8802252A431A80201C2A1C0C490D4B83
:102E50009847291C201C0C4B9847201C01210B4B28
:102E60009847C023AB40F2581202120AF2507FBDBD
:102E7000C40A002000140040190D000000E100E029
:102E800061290000110E0000490E0000ED0D000048
:102E9000F0B5294B85B09847284B1A7DD007FBD554
:102EA000274F69463A88274E0A81274A11886A4681
:102EB0005181318803AA1180244A11886A46D18140
:102EC000029907220A40012A31D01A8BD00530D44A
:102ED00059688022D2020A4301915A601A8B202538
:102EE000FF352A431A831A4C1A4ADC611A80197D6D
:102EF000124AC807FBD5108B284310831648D461AB
:102F00001080197D01200D4A0142FAD0138B1D4318
:102F10001583D461029B0724634018430290029BEF
:102F20003B6003980D4B30601380019951600C4B4E
:102F3000984705B0F0BDC04629230000004000417D
:102F40000040800004408000024080000640800075
:102F50000020400005A5FFFF44A5FFFF06A5FFFFD9
:102F60005D23000008B58022214B92029A618022E5
:102F700012059A611F4B08221A601F4B1A7852B231
:102F8000002A03DB1A7802218A431A701B4B1A7835
:102F9000D10611D41B789A060ED48023DB01188841
:102FA00017491A1C884207D01B6883F30888154B01
:102FB0009A60154B1B689847144B01221A70BFF397
:102FC0005F8F62B6124B9847124B9847124B984747
:102FD000124B9847124AC1239B00D058802100020F
:102FE000000AC9050143D1500E4B98470E4BFCE730
:102FF0000044004198440041001000403804004063
:10300000FFFF000000ED00E004400000140100207C
:10301000CD280000112E0000E12D00004D08000019
:1030200000E100E0912E00003D2D000070470000FF
:1030300002B4714649084900095C49008E4402BC4B
:103040007047C04603B47146490840004900095A18
:1030500049008E4403BC7047002934D0012300226C
:1030600010B488422CD301242407A14204D2814207
:1030700002D209011B01F8E7E400A14204D2814217
:1030800002D249005B00F8E7884201D3401A1A4394
:103090004C08A04202D3001B5C0822438C08A042CB
:1030A00002D3001B9C082243CC08A04202D3001B81
:1030B000DC082243002803D01B0901D00909E3E7FB
:1030C000101C10BC7047002801D00020C04307B47A
:1030D000024802A14018029003BDC046D90000007A
:1030E0000029F0D003B5FFF7B9FF0EBC4243891A9F
:1030F0001847C046002941D010B4041C4C40A446D7
:1031000001230022002900D54942002800D5404271
:1031100088422CD301242407A14204D2814202D246
:1031200009011B01F8E7E400A14204D2814202D266
:1031300049005B00F8E7884201D3401A1A434C0863
:10314000A04202D3001B5C0822438C08A04202D399
:10315000001B9C082243CC08A04202D3001BDC08C1
:103160002243002803D01B0901D00909E3E7101C02
:103170006446002C00D5404210BC7047002806D0A1
:1031800003DB0020C043400801E08020000607B4B4
:10319000024802A14018029003BDC0461900000079
:1031A0000029EBD003B5FFF7A7FF0EBC4243891AF5
:1031B0001847C0467047C04670B50E4B0E4D0024F0
:1031C000ED1AAD101E1CAC4204D0A300F358984772
:1031D0000134F8E700F036F8084B094D0024ED1AE9
:1031E000AD101E1CAC4204D0A300F3589847013424
:1031F000F8E770BD5032000050320000503200003D
:103200005432000010B50023934203D0CC5CC45468
:103210000133F9E710BD031C8218934202D01970E4
:103220000133FAE7704730303444000003020100F4
:103230000400080070008000010000010002030C7F
:1032400010600000F8B5C046F8BC08BC9E46704748
:10325000D9000000F8B5C046F8BC08BC9E467047CF
:04326000B1000000B9
:103264006D0400003D010000590100005D010000F3
:1032740051030000610100002D010000E101000084
:103284005D0100000000000041726475696E6F20EA
:103294004D300041726475696E6F2073726C202822
:1032A4007777772E41726475696E6F2E6F72672916
:1032B4000000000000030000000000000000000007
:1032C40000000000000000000000000000000000FA
:1032D40000000000000000000000000000000000EA
:1032E40000000000000000000000000000000000DA
:1032F40004030904050F0C0001071002020000007A
:10330400BC000020B4000020940000201400002021
:1033140000000020D0000020AC00002012010102B7
:1033240002000040032A4E000001010203010000D4
:1033340009024300020100C0320904000001020234
:1033440001000524001001042402020524060001E2
:10335400052401030107058303400010090401004B
:10336400020A00000007058102400000070502026E
:0C337400400000000100000000400000CC
:04000003000028F5DC
:104000000080002035430000FB410000FB41000020
:1040100000000000000000000000000000000000A0
:10402000000000000000000000000000FB41000054
:104030000000000000000000FB410000E94100001A
:10404000FB410000FB410000FB410000FB41000080
:10405000FB410000FB410000FB410000E14B000080
:10406000FB410000D5490000FB410000FB4100007E
:10407000FB410000FB410000E5490000FB4100005E
:10408000FB410000FB410000FB410000FB41000040
:10409000FB410000FB410000FB410000FB41000030
:1040A000FB410000FB410000FB410000FB41000020
:1040B00010B5064C2378002B07D1054B002B02D0FE
:1040C000044800E000BF0123237010BD2C00002035
:1040D00000000000086A000008B5084B002B03D060
:1040E0000748084900E000BF07480368002B03D0D9
:1040F000064B002B00D0984708BDC04600000000CA
:10410000086A0000300000202800002000000000A5
:1041100008B50D20012100F09FF908BD10B5FA2463
:104120000121A4000D2000F043FA201C00F04CF8FF
:1041300000210D2000F03CFA201C00F045F810BDD5
:1041400038B5134D1349281C00F074FA124913486E
:1041500000F070FA1249134800F06CFA1249134843
:1041600000F068FA1249134800F064FA124C13493F
:10417000201C00F05FFA291C00220123104800F0E7
:104180008FFB211C242223230E4800F089FB38BD1D
:104190000C01002000080042000C00421001002029
:1041A0000010004214010020001400420801002009
:1041B00000180042180100201C010020001C0042D1
:1041C00048000020A800002070B5041E08D0054B50
:1041D0001D681E1C00F010F833685B1BA342F9D960
:1041E00070BDC04620010020024B1A6801321A60DF
:1041F0007047C046200100207047FEE730B5404BB5
:104200001E225968082091430222114359603D49FA
:104210008B6903438B613C483C4B9882988A0243EC
:104220009A82DA689007FCD5394A0120107010781C
:10423000C40704D53648407840B20028F7DB012097
:104240009060507840B20028FBDB324C304844602C
:10425000507840B20028FBDB82242D48E4014480E2
:10426000507840B20028FBDB988C8024A0439884CF
:10427000D868C506FCD5284C2448C462DC682348AD
:10428000E506FBD5848C254D2C438484DC681F48CF
:10429000E506FBD5848C02252C438484D86804066B
:1042A000FCD51A48C0684506F8D5D868C406FCD5C0
:1042B00000209060507840B20028FBDB184C144876
:1042C00044605478124864B2002CFADB1D6A154C25
:1042D0002C401C621C6A8025AC431C620323836053
:1042E000114B436053785BB2002BFBDB00230B7256
:1042F0000E4A4B728B72CB720D4B1A6030BDC046AA
:1043000000400041000400400C060000000800408E
:10431000000C004001050100B805FF7D040A000003
:1043200000070300FFFCFFFF03060100006CDC0236
:104330000000002038B51049104CA14206D101F010
:10434000A5FFFFF75BFF00F059F90BE00C4D8D4224
:10435000F5D00023CA18E818A24204D2006804333A
:104360001060F7E7FEE79042E9D0064B064A934219
:10437000E5D2002204C3F9E7000000202C00002051
:10438000286A00002C000020AC050020264BFA21F2
:10439000186810B5890001F0CBF9244B0138984218
:1043A0001DD8234B234A5860106AC0210002000A1E
:1043B000090601431162002407229C601A601E4B0B
:1043C000FC211A6A0A431A62196AFF2212020A437E
:1043D0001A62196AA022D2020A431A6200E0FEE7BA
:1043E000201C0021013400F037F8132CF8D1134BB6
:1043F000134AA0215380134BC900998012491961B7
:104400001121997002215970187801431970597E51
:10441000C9090129FBD00D4B53800D4B41225A7025
:104420000C4A1A8110BDC04600000020FFFFFF00AB
:1044300010E000E000ED00E0000400401E4000003D
:10444000000C0040004000420018000F2140000016
:1044500000480042FF03000070B518244443204B7D
:1044600008261A1996571D1C013638D0012919D073
:1044700000290AD0022932D1E3561A495268DB01D9
:104480005B1899184031062007E0E3561549526839
:10449000DB015B189918403102200870012191401E
:1044A00059601CE0182811D0182358432B560D4989
:1044B00028184268DB015B189918403108780224FB
:1044C000A043087001219140996008E0064B022149
:1044D0001A780A431A70DA79D209FCD1E4E770BD80
:1044E0001463000000440041004800421822424387
:1044F000F8B52D4D0824AA181457031C621C50D07F
:10450000481C00240C284CD801F008F9071E1E1E78
:104510001E1E1E1E1E0A0A0A0A000124644240E0F2
:10452000092902D1181C002103E00A2904D1181C12
:104530000221FFF791FF23E000240B2931D1181C41
:104540000121FFF789FF2CE018225343EA18526833
:10455000EB560120141C04405508DB01002C11D03F
:10456000124C1B195D1930352E780C010F2131408A
:1045700021439A18C9B22970403213781843107039
:1045800000240EE0094E0F279B195D1930352E7857
:104590009A18BE433143C9B2297040321378184388
:1045A0001070201CF8BDC046146300000044004198
:1045B000182358430E4A30B5131808241C570134E9
:1045C00015D080560B4C5B68C0010219D4184034DA
:1045D00004252570002904D0012908D19940916152
:1045E00005E001229A40131C034A8018436030BD45
:1045F00014630000004400411044004110B5FFF76F
:10460000C5FE0120FFF7E0FD084C201C00F0B2FAC7
:10461000201C00F09DFAFFF77BFDFFF77FFD044BA8
:10462000002BFAD000E000BFF7E7C0462C010020C5
:104630000000000001607047F7B508AC26780468F8
:104640009D1E27686C1EA541ECB2920705683A438F
:1046500027063A432A600268072529405068B501B9
:10466000002C00D05C03294301430C435460F7BD88
:1046700030B50368C0251C68AD0312052A402243EB
:10468000C024A402090421401143196003685A6838
:1046900014435C6030BD036801211A680A431A6044
:1046A0000268116801231942FBD1D1691942F8D17E
:1046B0007047036802211A680A431A600268D369C6
:1046C0009907FCD470470268137ED907FCD5704760
:1046D000036800225A8370470368187E4007C00FA2
:1046E00070470368588B4007C00F70470368588BAA
:1046F0008007C00F70470368588B0123184070472C
:104700000368188DC0B2704738B5041C0D1CFFF744
:10471000DAFF236801201D8538BD000002682349A7
:1047200030B58A4210D022498A4210D021498A42AB
:1047300010D021498A4210D020498A4210D0204905
:104740008A4210D0002210E0092314220DE00A232F
:1047500015220AE00B23162207E00C23172204E09F
:104760000D23182201E00E23192258B2012484409F
:104770001449800880000C6040180325C02189007E
:104780002B40AB404458FF259D40AC43C0259D4085
:104790002B1C234343508023DB011A430A4B5A80CE
:1047A0005A7852B2002AFBDB30BDC04600080042F6
:1047B000000C0042001000420014004200180042A9
:1047C000001C004200E100E0000C0040F8B5041CB1
:1047D000151C0F1C1E1CFFF75EFF201CFFF79EFF21
:1047E000B9001C220A4069072368090C0A431A60B1
:1047F000226884239375012F26D11020002D03D029
:104800000320022D00D1082001F0DAFB051C301C2A
:1048100001F0D6FB011C281C01F018F90B4B051CFC
:10482000186801F0CDFB011C281C00F0E9FF011CF9
:10483000FE20800501F034FA054901F007F900F087
:10484000C7FF246880B2A081F8BDC04600000020E8
:1048500000FF7F470120704710B5041C0069FFF777
:104860001AFF201C143000F06CFD10BD08B5006963
:10487000FFF729FF08BD08B5143000F074FD08BD2E
:1048800008B5143000F075FD08BD08B5143000F00F
:104890005CFD08BD08B50069FFF736FF012008BDC3
:1048A000F8B51D1C00234360FA239B008360084B6E
:1048B000041C0833036014300F1C161C00F02BFD81
:1048C000231C5C332761201C1E705D70F8BDC04640
:1048D0009867000010B5041C0069FFF7FDFE002872
:1048E00007D02069FFF70CFF011C201C143000F0DA
:1048F0001DFD2069FFF7F5FE002809D12069FFF7AB
:10490000F5FE002804D12069FFF7F5FE002802D04B
:104910002069FFF7DDFE10BD0F23081C98433038D7
:10492000434258417047002070470F231940012926
:1049300005D002394B424B410220C01A00E0002052
:1049400070470000F0B5031C85B003915C33041C74
:10495000182718783B1C43431A4E0821F318595660
:10496000151CFFF7C3FD231C5D331878082147434E
:10497000F6197156FFF7BAFD039B00222069012149
:10498000FFF724FF291C201CFFF7CDFF291C071C63
:10499000201CFFF7CAFF291C061C201CFFF7BCFFC8
:1049A000331C0090391C20690122FFF745FE206965
:1049B00001210322FFF75CFE2069FFF77AFE05B0B4
:1049C000F0BDC0461463000008B51322FFF7BAFF1C
:1049D00008BD000008B50248FFF77CFF08BDC046CF
:1049E0004800002008B50248FFF774FF08BDC04624
:1049F000A800002008B500F03FFC08BDF8B5124B38
:104A0000061C1B680D1C171C002B02D101246042E0
:104A100019E000F031FC041EBC4200D93C1C2F19E7
:104A2000BD4205D0301C00F0E1FB28700135F7E7EE
:104A3000002C07D0301C00F01FFC002802D1301CD5
:104A400000F024FC201CF8BD3801002013B56C4692
:104A50000734211C0122FFF7D1FF012801D1207862
:104A600001E00120404216BD38B5104B051C1B6803
:104A7000141C002B15D000F099FB08350C4A6B0173
:104A80009B18DA7902210A43DA715979802252425D
:104A90000A435A71064A6B019B18DB799A07F9D5CC
:104AA00002E00120404200E0201C38BD3801002017
:104AB00000500041F8B50F1C161C141C0025002CDA
:104AC00007D07919221C002000F070FB2D18241A41
:104AD000F5E7301CF8BD30B50123A1B0C218013A8A
:104AE00014785A00002C0CD1C0239B001343694654
:104AF00000200B80FFF7DEFF431E9841C0B221B0BB
:104B000030BD8D1A002DEFDD6D46AC520133E5E767
:104B100008B50279002A04D100F0A6FC002809D1CA
:104B200006E00023022A06D100F01AFD002801D079
:104B300000F09CFA0123181C08BD10B5041C00F0FD
:104B40009BFB002802D0201C00F0AAFB10BD000037
:104B5000064B10B51B680024A34204D000F07AFA7B
:104B6000034B1C600124201C10BDC04628010020FE
:104B70003801002008B500F0D7F9024B01221A6075
:104B800008BDC0462801002008B502280CD1A22388
:104B9000114A40215B00D15400F06EFB002819D06F
:104BA0000E4800F02FFC15E0032806D10A4BB22274
:104BB000520080219954682207E001280AD1064B4F
:104BC00092225200802199542822FF32995C0220BF
:104BD0000143995408BDC0460050004184040020A0
:104BE000F0B5B24CA9B0268C1025F6B2002E1BD120
:104BF0002023A582A3820123A382A38B08273B4203
:104C00000AD08023A372301C311C00F037FAA84B65
:104C10009D72A84B1E60A783228B04231A4200D1E9
:104C20007BE1A24A938378E1A14B1A7AD2B2029235
:104C30002A4200D159E11D72002004A900F00AFBAC
:104C40009B4840234371049B60201D78284000D07E
:104C500024E15A78002A0CD108A9002D03D10D7047
:104C60004D70281C14E0944B1B78012B0BD00A705C
:104C70000CE0012A11D19B78012B0BD18F4B08A995
:104C80001B78012B01D10B7000E0087000204870E8
:104C90000222F8E0884B1870FDE0032A11D19A78BF
:104CA000012A05D1854B08A91A70087000F07EFA18
:104CB00004998B78002B00D0F5E07F4B01221A700D
:104CC000E9E0052A03D1987800F0F4FAEBE0062A2F
:104CD00000D0ABE0DD78022D60D1DB88019300F0DD
:104CE000BDFB071C00F0BEFB041C00F017FC001904
:104CF000039000F0B7FB041C00F010FC019A24188C
:104D00000934A24207D900F0ADFB041C00F006FCF8
:104D100024180934019405AD0924221C281C002103
:104D200001F0E3FA2C70039C02226B465A75093499
:104D30006B46DC82032206AB1A7001226B465A7660
:104D4000C0226B46DA7608ACFA2307AA1370221C3D
:104D500003CD03C20025137000F084FB854205D209
:104D60007A5D631901355A72EDB2F5E700F0D2FBB6
:104D70000025071C00F0D2FB854208D200F072FB30
:104D80007B5D6219101801354372EDB2F2E7019AAA
:104D9000802A00D980220020211C44E0222D02D14B
:104DA00000F0C0FB18E0212D1AD108AC0927002122
:104DB0003A1C201C01F099FA0123A370E37063717F
:104DC000222327706570A37100F0AAFB211CE071FB
:104DD0003A1C0020FFF76EFE431E9841C0B260E00F
:104DE000012D04D1DA883649112A1AD816E0032D8C
:104DF00070D19A78002A05D13249DA880B7893422B
:104E00000CD80EE0022A02D1D9882F4803E0012AEB
:104E100060D1D9882D48FFF75EFE42E0D2B2002A69
:104E200000D10A780020FFF745FE3CE0072A51D068
:104E3000082A02D100201F4924E0092A1ED1EA06CF
:104E400048D10420832100F019F90120822100F0CB
:104E500015F90220011C00F011F90320832100F054
:104E60000DF9049B9A78134B1A602A230222FF3310
:104E7000E2544A230122FF33E2540CE00A2A05D10E
:104E800013490020012200F091F90CE00B2A0AD10D
:104E90009A780F4B1A6000F0E9F804E0181CFFF74D
:104EA00037FE002816D000F07BF916E000500041D4
:104EB000FF5000413801002024010020340100206F
:104EC000E4670000E0670000C8670000D3670000E7
:104ED00030010020002000F0C5F90298402318425C
:104EE00003D00F490B7220234B7101239E430024F2
:104EF000E0B2002E11D0331C2341DA070AD509494C
:104F000063015B18DB799A0701D0FFF73DFE0123AF
:104F1000A3409E430134092CEAD129B0F0BDC0461C
:104F2000FF5000410051004130B53E4B2021DA696D
:104F300001200A43DA613C4B06241A7802431A70B6
:104F40003A4B0F221978914319701978214319703F
:104F500037490C782043087019780A401A701A787B
:104F600060210A431A70334B334A5A805A7852B23E
:104F7000002AFBDB314B01211A780A431A70997819
:104F80002E4AC807FBD41178022001432C48117027
:104F90000268510B1F221140914200D1052111409E
:104FA0008C011D8D27492940214319850468A10CD6
:104FB0000A401F2A00D11D221C8D1F210A408C434C
:104FC00022431A8502680721D20D0A408A4200D185
:104FD00003220A40188D11031B4A02400A431A8516
:104FE00019787F220A401A701A7804210A431A702D
:104FF000164A0C205A621989814319810023D1185D
:10500000002008602033802189018B42F7D1104BAA
:10501000C122920099580902090A995080221A6007
:1050200030BDC04600040040584400413C440041AB
:1050300059440041000C004006400000005000416F
:10504000246080003FF8FFFFFF8FFFFFAC040020CB
:1050500000E100E0044B01211A898A431A810822E9
:105060001A8304221A83704700500041024B5A6988
:10507000920B92035A617047AC040020F0B583296B
:1050800011D1021C3F4B083252014021D1543E4AFB
:105090004301D3185C693D493D4AC00121401018C5
:1050A000596118616DE002291FD13A4B4201364C1B
:1050B000D11803234B70A3185E68344D800135402E
:1050C000C026B60535435D60334D28181051586829
:1050D000324A02408020400302435A605A68920BD1
:1050E00092035A6040234B714BE0822914D1294C22
:1050F00042011319302159702349244C8A185569EB
:1051000023492C40C025AD05C0012C43081854612B
:10511000106180225A7134E0002932D11D494001CA
:1051200042181123184D8024537064424023937118
:1051300054712B185968154F4900490859605E6928
:105140001549760076085E615E683E40B446C0262A
:10515000B605644634435C605C6927403E435E614B
:10516000415158680D4901408020C00201435960F7
:105170005968890B89035960802340215B429171F2
:105180005371F0BD00500041AC040020FFFFFF8FC1
:105190003C010020FF5000413C030020FF3F00F095
:1051A000014B80229A717047FF50004170B50C4D41
:1051B000C301ED18061C281C141C01F08DF8094BC6
:1051C00076019E1935617169074A201C0A40726197
:1051D0007269A104920B890C92030A43726170BD3B
:1051E0003C010020AC040020FF3F00F070B5134CE0
:1051F000134A8101430165189D50D2185668114D1C
:1052000035408026B602354355605568AD0BAD0379
:1052100055600D4A9D180D4A9B1840225A712B1C4F
:10522000FF331A7A01231A42F9D0094A4001801843
:10523000C2791343C371605C70BDC0463C0300205B
:10524000AC040020FF3F00F000500041FF5000413F
:1052500000510041024B8001181808607047C04699
:105260003C030020034BC0B24001C018202343710F
:105270007047C04600510041034B40011818406878
:105280008004800C7047C046AC040020034B4001F2
:10529000C01840234371012303727047FF5000413F
:1052A000034B4001C01880238371022303727047AF
:1052B000FF5000410C4B02215A69920B92035A6134
:1052C0000A4B1A7A0A431A729979802252420A4387
:1052D0009A711A7A9107FCD580235B421843044BDC
:1052E000C0B298727047C046AC040020FF50004125
:1052F00000500041F8B5061C0C1C8F180025BC425C
:1053000007D0336821781B68301C984701342D186A
:10531000F5E7281CF8BD10B500214022041C00F060
:10532000E4FF0023201C2364636410BD026C10B5ED
:105330003F23541C2340446CA34201D08154036496
:1053400010BD0023036443647047436C026C9342B6
:1053500006D0C25C3F2101330B404364101C01E0C6
:10536000012040427047026C436CD01A00D5403097
:105370007047436C026C934201D0C05C01E0012095
:1053800040427047034B186C5B6CC01A3F231840B7
:105390007047C0463C040020054B196C5A6C914282
:1053A00002D05A6C985C01E0012040427047C04630
:1053B0003C04002013B502686B46D971073354686A
:1053C000191C0122A04716BD38B50D4B041C196CE1
:1053D0005A6C914211D05A6C3F219D5C5A6C02204C
:1053E00001320A405A64FFF705FB002803D0236806
:1053F000201C9B699847281C01E00120404238BDD1
:105400003C04002038B50C4D2C6C3F2301341C406B
:105410006B6C9C420FD00220FFF7ECFA002803D1FE
:105420000220FFF733FF06E00220FFF70FFB2B6C93
:105430002C64E854E9E738BD3C04002008B503209B
:10544000FFF77BFB08BD10B5041C0320FFF70CFB26
:10545000002801D10123636010BD0000004870479F
:10546000206800004220704710B50278041C437881
:10547000A12A08D1212B2CD1002017490722FFF7A0
:1054800019FB012026E0212A23D1202B0DD1002059
:10549000FFF7F2FE0E28FAD90023E218117A0E4A1D
:1054A00099540133072BF8D113E0222B11D18278C4
:1054B000094BDA7119689622D200914209D1DC7940
:1054C00001231C4003D1FA2000F016F901E000F09E
:1054D0001DF9002010BDC04604000020044B00222E
:1054E0005A60FA2292009A60024A08321A607047A3
:1054F00084040020F8670000036870B59B68041CF2
:105500000D1C98472368061C291CDB68201C984743
:10551000F0B270BD0048704708690000192070475C
:105520006520704708B5002002496522FFF7C2FADE
:1055300008BDC0462169000013B56B461870141CE5
:1055400000235A1CA34206D0131C8A18013A127871
:105550006846C254F5E769460420FFF785FA13BD93
:1055600008B50178031C4278A1290ED10223101C32
:105570009843012817D000209A4214D10A490122E9
:10558000FFF714FEFFF70CFE0CE0002021290AD1E2
:105590000B2A02D19A78054B03E00A2A03D1DA7864
:1055A000014B1A70012008BD0D0000200C000020E6
:1055B00008B502200822FFF7BFFF08BD10B58729F4
:1055C00002D97831C9B218E04BB2002B08DA803921
:1055D00001238B40191C037A1943017200210CE04E
:1055E000194B595C00292BD04BB2002B05DA037AFA
:1055F0000222134303727F231940837A8B4219D00E
:10560000C37A8B4216D0037B8B4213D0437B8B42F1
:1056100010D0837B8B420DD0C37B8B420AD00023FA
:10562000C218947A002C01D1917203E00133062B49
:10563000F6D105E0011C0831FFF7BAFF012002E0B6
:1056400001234360002010BD8868000010B5872941
:1056500002D97831C9B219E04BB2002B08DA80398F
:1056600001238B40191C037A8B43037200210DE048
:10567000114B595C002399421BD04BB2002B05DA29
:10568000037A0222934303727F231940031C0622EC
:10569000002904D09C7A8C4201D100249C72013AEA
:1056A000D2B20133002AF3D1011C0831FFF780FF89
:1056B0000123181C10BDC0468868000008B5011CF5
:1056C00000238372C372037343738373C3730372C0
:1056D0000831FFF76DFF08BD044B00221A70044B20
:1056E0005A60044A08321A607047C0469804002085
:1056F0009C0400206868000008B5024B1860024B4B
:105700009847C046100000200D6A0000024B01229D
:1057100052421A607047C0461000002002B4714621
:1057200049084900095C49008E4402BC7047C046E4
:10573000002934D00123002210B488422CD3012444
:105740002407A14204D2814202D209011B01F8E7D9
:10575000E400A14204D2814202D249005B00F8E792
:10576000884201D3401A1A434C08A04202D3001BBE
:105770005C0822438C08A04202D3001B9C082243F1
:10578000CC08A04202D3001BDC082243002803D02F
:105790001B0901D00909E3E7101C10BC7047002861
:1057A00001D00020C04307B4024802A14018029073
:1057B00003BDC046190000000029F0D003B5FFF773
:1057C000B9FF0EBC4243891A1847C0467047C0460D
:1057D0009E2110B5C905041C00F072FC002803D1FD
:1057E000201C00F0CDFB10BD9E21C905201C00F03F
:1057F00057FA00F0C5FB80231B06C018F3E7C0462C
:10580000F0B55F4656464D464446F0B44602450064
:10581000C00F85B00F1C760A2D0E804641D0FF2D9B
:1058200026D08024240400212643F6007F3D8946AB
:105830008B46F90F7C027800640A000E00918A46BC
:105840003CD0FF2834D080231B041C430023E400F9
:105850007F380193009F4346019A7B4049469C460E
:1058600011430F2900D971E0764F89007F58BF4658
:10587000002E3ED10822022391469B46D9E75A4684
:10588000341CC24601920199022937D0032900D164
:10589000CFE0012900D0ABE053460B4000220026A8
:1058A00032E0002E19D10421012289469346C0E737
:1058B000221C531E9A4102320192CBE70127019725
:1058C000002CC7D0201C00F005FC431F9C40762311
:1058D0005B420021181A0191BCE7301C00F0FAFB72
:1058E0007625431F9E406D4200232D1A99469B4604
:1058F0009FE70C23032199468B469AE7D446012360
:1059000067463B40FF2200267602D205700ADB077D
:105910001043184305B03CBC90469946A246AB469E
:10592000F0BD80260023F603FF22EDE700220026CB
:10593000EAE78020C00306423BD0044239D1061C6E
:1059400026437602760A009BFF22DDE7281A0390A1
:1059500076016401A64239D3361B1A2201230120A5
:10596000311C5B007600002901DBB44201D8361BF4
:105970000343013A002AF3DC741EA641341C1C4385
:10598000039A7F32002A27DD630704D00F232340C8
:10599000042B00D00434270103D52B4B039A1C4061
:1059A0008032FE2A0BDD012361460B40FF220026D8
:1059B000AAE706437602760A4346FF22A4E7A4013B
:1059C00001236746660AD2B23B409DE7039F1B2234
:1059D000013F03970023C2E77E23039F5B42DB1B4B
:1059E0001B2B07DD012361460B40002200268BE7BD
:1059F000D446C5E7221CDA40039B9E339C40231CFF
:105A00005C1EA34113435A0704D00F221A40042AF4
:105A100000D004335F0105D5012361460B4001220C
:105A2000002671E79E01624601231340760A002298
:105A30006AE78026F60326437602760A5346FF225B
:105A400062E7C04688690000FFFFFFF7F0B55F46D8
:105A500056464D464446F0B44402460083B00F1CFF
:105A6000640A360EC50F002E41D0FF2E22D08023AF
:105A70001B0400201C43E4007F3E82468046391C04
:105A80004B007F02C90F7F0A1B0E8B463BD0FF2BBA
:105A900034D0802212041743FF007F3B00215A4676
:105AA0006A40019252460A430F2A63D87A4892000C
:105AB00082589746002C3FD10822022392469846EE
:105AC000DDE70195404602282AD1019A01251540BB
:105AD000FF2300246402DB05600AED071843284316
:105AE00003B03CBC90469946A246AB46F0BD002CA4
:105AF00027D10420012282469046C0E7391C4A1E65
:105B000091410231CBE70121002FC8D0381C00F0B1
:105B1000E1FA431F9F4076235B421B1A0021BEE738
:105B2000032800D1AEE001284FD101984246104031
:105B3000C5B200230024CDE70C2303209A468046FB
:105B40009DE7201C00F0C6FA7626431F9C40764253
:105B50000023361A9A46984691E780240025E403EC
:105B6000FF23B7E75B463C1C01938846AAE73C1C31
:105B70008846A7E7250C24043A0C240C3F04F618A9
:105B80003F0C211C231C794353436F435543FB189F
:105B90000A0C9B18B1469F4202D980225202AD18CE
:105BA00009041A04090C521894011B0C611E8C4143
:105BB000920EED181443AD012C43230105D50122AB
:105BC00063080120144081441C434B467F33002B63
:105BD0002DDD600704D00F222240042A00D00434B7
:105BE000220103D52D4B1C404B468033FE2B17DD85
:105BF000019B01251D400024FF236BE78020C0038B
:105C0000044208D0074206D1041C3C436402640AE3
:105C10005D46FF235EE704436402640AFF2359E7FD
:105C20000198A4010125640ADBB2054052E77E23F6
:105C30005B424A469B1A1B2B05DD019B01251D403B
:105C40000024002346E7221CDA404B469E339C404A
:105C5000231C5C1EA3411343580704D00F221A4093
:105C6000042A00D004335A0105D5019B01251D40AB
:105C7000002401232EE701989C010125640A0540B8
:105C8000002327E78027FF03019B3C436402012593
:105C90001D40640AFF231DE7C8690000FFFFFFF7EE
:105CA000F8B5C20F430244004D024800240E161CF2
:105CB0009B09000EC90FAD09FF2800D17EE0012726
:105CC00079408A4258D0221A002A00DC89E0002854
:105CD0001BD1002D00D075E0580704D00F221A40C8
:105CE000042A00D00433590138D50134FF2C00D1E7
:105CF00083E09B0101225B0AE0B232405B02C405F3
:105D0000580AD20720431043F8BDFF2CE4D080216D
:105D1000C9040D431B2A00DD2DE1291C2020D140A0
:105D2000821A95406A1E95410D435B1B5801D3D5DD
:105D30009B019F09381C00F0CDF9421F9740944207
:105D400060DC141B1F231B1B3A1C9F40611C3B1C67
:105D5000CA405F1EBB4113430024BDE70122DB089C
:105D6000E0B23240FF2C04D1002B7ED08021C90349
:105D70000B435B025B0AC1E7211A002946DD0028BC
:105D800026D0FF2CA8D08020C00405431B2900DDAD
:105D9000EFE0281C2027C840791A8D40691E8D41EC
:105DA00005435B19590197D50134FF2C5CD0734929
:105DB00001221A400B405B0813438DE7002D00D0F1
:105DC0007FE77CE7013A002AAFD0FF2CA2D183E71E
:105DD000002D00D180E701390029E2D0FF2CD5D178
:105DE0007AE7002A1ED1621CD2B2012A4EDD5F1B67
:105DF0007A0126D5EF1A0E1C9CE701223240FF20C3
:105E000000237BE75D4BA41A3B4065E7002946D1A0
:105E1000611CC8B201282ADDFF2925D0EB185B08D8
:105E20000C1C59E7002C13D0FF2818D08024E40460
:105E3000524223431B2A4DDD0123EB1A041C0E1C86
:105E400074E7002F00D075E700220020002390E7C0
:105E5000002B3BD0D243002AEFD0FF28EAD12B1CE5
:105E6000FF240E1C38E70022FF20002346E7002C09
:105E70005AD1002B77D0002D00D12DE75B195801A6
:105E800000D429E73D4A0124134025E7002C15D111
:105E9000002B2FD1002DD7D02B1C0E1C1CE7002C63
:105EA00021D1002B53D0C943002904D0FF284BD067
:105EB0001B294FDD01235B19041C73E7002B22D142
:105EC000002DD0D02B1C0E1CFF2405E72B1C041C1E
:105ED0000E1C01E71C1C2026D440B21A93405A1E07
:105EE00093412343A9E7FF282ED08024E4044942AC
:105EF0002343DDE7002D00D1EEE65A1B500134D5D7
:105F0000EB1A0E1CE8E6FF24002D00D1E4E6802207
:105F1000DB08D203134204D0ED08154201D12B1C3B
:105F20000E1CDB00FF24D7E6002B0DD0FF24002D34
:105F300000D1D1E68022DB08D2031342F1D0ED0874
:105F40001542EED12B1CECE72B1CFF24C4E62B1CC6
:105F5000041CC1E61C1C2027CC40791A8B40591E1A
:105F60008B412343A7E72B1CB6E6131E00D0B3E6F4
:105F70006AE7012515E70125D7E6C046FFFFFFFBCD
:105F80004302590A4300C20F1B0E00207E2B0DDD79
:105F90009D2B0CDC802000040143952B0ADC96200D
:105FA000C31AD9404842002A00D1081C7047034B4D
:105FB000D018FBE7963B9940F4E7C046FFFFFF7F10
:105FC00010B5041E33D000F085F89E231B1A962BC3
:105FD00009DC083884406402640ADBB26402DB0531
:105FE000600A184310BD992B0ADD0522121A211CE4
:105FF000D1400A1C011C1B318C40611E8C41144392
:10600000052801DD421F9440144A2240610704D054
:106010000F210C40042C00D0043251010AD59F23DB
:10602000181AFF2816D09401640AC3B2D6E70023D9
:106030000024D3E7D208FF2B03D05402640ADBB25A
:10604000CCE7002A06D08024E40314436402640AE7
:10605000FF23C3E7FF230024C0E7C046FFFFFFFB89
:106060008446081C6146FFE71FB500F0C3F800280E
:1060700001D40021C8421FBD10B500F049F84042CC
:10608000013010BD10B500F0B5F8002801DB00208C
:1060900010BD012010BDC04610B500F0ABF80028BF
:1060A00001DD002010BD012010BDC04610B500F07C
:1060B00059F8002801DC002010BD012010BDC046A9
:1060C00010B500F04FF8002801DA002010BD0120C3
:1060D00010BDC0461C2101231B04984201D3000CB3
:1060E00010391B0A984201D3000A08391B0998424B
:1060F00001D30009043902A2105C40187047C04661
:106100000403020201010101000000000000000080
:106110004A02430270B55C0A550A43004A001B0E4E
:10612000C60F120EC90FFF2B05D0FF2A08D0012081
:1061300093420BD070BD0120002CFBD1FF2AF6D179
:106140000120002DF6D101209342F3D1AC42F1D1D0
:106150008E4205D0002BEDD1201C441EA041E9E762
:106160000020E7E74A024302F0B55C0A550A430003
:106170004A001B0EC60F120EC90FFF2B31D0FF2A8B
:1061800034D0002B16D1604260418446002A14D0DE
:10619000002820D18E4217D1934215DC04DBAC429B
:1061A00012D80020AC4212D270427041404201230A
:1061B00018430CE0002AEDD194466F426F416046CF
:1061C000002805D1002FE5D0704201231843F0BD0F
:1061D0000020002FFBD14842484140420123184390
:1061E000F5E7002CCBD002204042F0E7002DC8D0CC
:1061F000F9E7C0464A024302F0B55C0A550A43007B
:106200004A001B0EC60F120EC90FFF2B27D0FF2A04
:1062100029D0002B10D0002A15D194466F426F412F
:106220006046002815D00020002F04D14842484184
:10623000404201231843F0BD604260418446002A79
:10624000ECD00028F2D18E4211D0704201231843C5
:10625000F1E7002FF7D0704201231843EBE702204B
:10626000002CE8D1D3E70220002DE4D1D1E79342FE
:10627000EBDC04DBAC42E8D80020AC42DBD270425D
:106280007041404201231843D5E7C04670B50E4B1C
:106290000E4D0024ED1AAD101E1CAC4204D0A3001C
:1062A000F35898470134F8E700F028F8084B094DF7
:1062B0000024ED1AAD101E1CAC4204D0A300F3580C
:1062C00098470134F8E770BD140000201400002046
:1062D000140000202400002010B50023934203D0B6
:1062E000CC5CC4540133F9E710BD031C82189342FF
:1062F00002D019700133FAE770470000F8B5C046C4
:10630000F8BC08BC9E467047F8B5C046F8BC08BC4F
:106310009E467047000000000B00000002000000D5
:106320001C000000FF00FFFFFFFF0B00000000004B
:106330000A000000020000001C000000FF00FFFF38
:10634000FFFF0A0000000000080000000400000039
:106350001C000000FF000000000010000000000012
:1063600009000000040000001C000000FF00010004
:1063700001000900000000000E0000000400000001
:106380001C000000FF00000300030E0000000000DE
:106390000F000000040000001C000000FF000103CB
:1063A00001030F00000000001400000005000000C1
:1063B0001C000000FF0006000600040000000000B2
:1063C00015000000050000001C000000FF00070091
:1063D00007000500000000000600000004000000A7
:1063E0001C000000FF00000100010400000000008C
:1063F00007000000040000001C000000FF00010175
:10640000010105000000000012000000040000006F
:106410001C000000FF000003000302000000000059
:1064200010000000040000001C000000FF0000023B
:106430000002000000000000130000000400000043
:106440001C000000FF000103010303000000000026
:1064500011000000040000000C000000FF00010219
:10646000FFFF0100FF00000000000000FF0000002F
:1064700000000000FF00FFFFFFFFFF000000000022
:10648000030000000100000002000000FF00FFFF09
:10649000FFFFFF00000000001600000002000000E7
:1064A00004000000FF00FFFFFFFF060000000000E7
:1064B000170000000200000004000000FF00FFFFC2
:1064C000FFFF0700000000000C00000003000000B8
:1064D00004000000FF00FFFFFFFF0C00FF000000B2
:1064E00000000000FF00000000000000FF00FFFFB0
:1064F000FFFFFF00010000000B0000000300000090
:1065000004000000FF00FFFFFFFF0B000100000080
:106510000A0000000300000004000000FF00FFFF6D
:10652000FFFF0A00FF00000000000000FF00000065
:1065300000000000FF00FFFFFFFFFF00FF00000062
:1065400000000000FF00000000000000FF00FFFF4F
:10655000FFFFFF000000000002000000010000003B
:10656000020000000000FFFFFFFF0200010000002A
:106570000800000001000000020000000200FFFF10
:10658000FFFF0800010000000900000001000000FA
:10659000020000000300FFFFFFFF090000000000F1
:1065A0000400000001000000020000000400FFFFE2
:1065B000FFFF0400000000000500000001000000D3
:1065C000020000000500FFFFFFFF050000000000C3
:1065D0000200000001000000020000000A00FFFFAE
:1065E000FFFF020001000000030000000B0000009C
:1065F00004000000FF00FFFFFFFFFF00000000009D
:106600001B0000000B00000004000000FF00FFFF63
:10661000FFFFFF00000000001C000000060000005B
:1066200000000000FF00FFFFFFFFFF000000000070
:10663000180000000600000000000000FF00FFFF3F
:10664000FFFFFF000000000019000000060000002E
:1066500000000000FF00FFFFFFFFFF00010000003F
:10666000160000000300000000000000FF00FFFF14
:10667000FFFFFF0001000000170000000300000002
:1066800000000000FF00FFFFFFFFFF000000000010
:10669000160000000200000000000000FF00FFFFE5
:1066A000FFFFFF00000000001700000002000000D4
:1066B00000000000FF00FFFFFFFFFF0000000000E0
:1066C000130000000200000000000000FF00FFFFB8
:1066D000FFFFFF00000000001000000002000000AB
:1066E00000000000FF00FFFFFFFFFF0000000000B0
:1066F000120000000200000000000000FF00FFFF89
:10670000FFFFFF0000000000110000000200000079
:1067100000000000FF00FFFFFFFFFF00000000007F
:106720000D000000040000000C000000FF00050048
:10673000FFFF0D0000000000150000000500000034
:106740000C000000FF000700FFFFFF00000000003A
:1067500006000000040000000C000000FF00000123
:10676000FFFFFF0000000000070000000400000021
:106770000C000000FF000101FFFFFF00000000000F
:106780000200000001000000020000001400FFFFF2
:10679000FFFF0200000000000000000000000000F9
:1067A00095480000F5520000774800008B48000033
:1067B000814800006D480000C949000059480000A8
:1067C000554800000000000041726475696E6F203A
:1067D0004D300041726475696E6F2053726C000019
:1067E0000403090412011001EF020140032A4E8044
:1067F0000001010200010000000000000000000094
:10680000B55300004754000085530000C9530000F1
:10681000995300003D5400000554000000000000A2
:10682000080B00020202000009040000010202003D
:1068300000052400100104240206052406000105B9
:106840002401010107058103100010090401000261
:106850000A0000000705020240000007058302400D
:106860000000000000000000000000000000000028
:10687000F9540000F5520000BD5500004D560000CF
:10688000BD560000000000000000000000000000F5
:106890002A2B28000000000000000000000000007B
:1068A00000000000000000002C9EB4A0A1A2A434AF
:1068B000A6A7A5AE362D3738271E1F202122232458
:1068C0002526B333B62EB7B89F8485868788898AF4
:1068D0008B8C8D8E8F909192939495969798999A90
:1068E0009B9C9D2F3130A3AD350405060708090A8E
:1068F0000B0C0D0E0F101112131415161718191A70
:106900001B1C1DAFB1B0B50009040200010300005B
:1069100000092101010001226500070584034000F0
:106920000105010902A1010901A10085010509195B
:106930000129031500250195037501810295017553
:1069400005810305010930093109381581257F7555
:106950000895038106C0C005010906A1018502054D
:106960000719E029E71500250175019508810295B1
:106970000175088103950675081500256505071939
:106980000029658100C000004C590000FE5800003D
:106990002C590000865800002C5900002259000094
:1069A0002C59000086580000FE580000FE580000D8
:1069B00022590000865800007E5800007E580000D2
:1069C0007E58000032590000745B00006E5B0000CE
:1069D0006E5B0000645B0000C45A0000C45A0000F3
:1069E0005A5B0000645B0000C45A00005A5B000060
:1069F000C45A0000645B0000C25A0000C25A000082
:0C6A0000C25A0000FC5B00000000000017
:106A0C0072B6054B0F215A788A435A701A780221B4
:0C6A1C000A431A70FEE7C046001000405C
:106A280040420F0000C20100000008000101000000
:106A3800FFFFFFFFD940000041410000DD54000086
:0C6A4800D9560000B14000000000000022
:106A54000000000000000000000000000000000032
:106A64000000000000000000000000000000000022
:106A74000000000000000000000000000000000012
:106A84000000000000000000000000000000000002
:040000030000433581
:00000001FF
